:020000020000FC
:1000000010C040C040C040C040C064C064C066C0B2
:1000100066C03CC05DC05DC063C063C03EC13EC140
:100020003EC101E00EBF0FE50DBF02E000B90027A1
:100030000ABB00270BBB07E007BB08BB02E000BF01
:1000400005E003BF04EF06BF02E009BF01E003BD06
:1000500000270FBD05E00EBD10E001E61BBD0ABD87
:1000600002E00CB901E003BD00E007B900E103B90B
:1000700008EC06B90FEF0093600000E205BF78942A
:100080008895FECF18951895189518950F930FB76A
:100090000F9300918000002329F00A9500938000BF
:1000A00009F4C09A00918200002329F00A95009378
:1000B000820009F4C19A00918300002329F00A9577
:1000C0000093830009F4C29A0F910FBF0F91189506
:1000D000189518951895E8ECE6B91895189518959F
:1000E0001895C5B1D7B1D770E0916000EE2309F043
:1000F000ADC0D030B1F5F2E0E0E0EF0FE7B9EE27A8
:10010000E1B9EDE0EABBEE27EBBBEABBEFEFE1B90B
:10011000C0936800C695C695E09170001E2EE695C6
:10012000E6951E1A1C0EE12DE0937000F091780008
:100130001F2EF695F695F6951F1AC6951C0EF12DF5
:10014000F0937800EF1BE2302CF0C098F3E0F093CE
:10015000800005C0F0918000FF2309F4C09AC2E03E
:1001600098C0D230B1F5F3E0E0E0EF0FE7B9EE2749
:10017000E1B9EDE0EABBEE27EBBBEABBEFEFE1B99B
:10018000C0936A00C695C695E09172001E2EE69552
:10019000E6951E1A1C0EE12DE0937200F0917A0094
:1001A0001F2EF695F695F6951F1AC6951C0EF12D85
:1001B000F0937A00EF1BE2302CF0C198F3E0F0935B
:1001C000820005C0F0918200FF2309F4C19AC3E0C8
:1001D00060C0D330B1F5F0E0E0E0EF0FE7B9EE2713
:1001E000E1B9EDE0EABBEE27EBBBEABBEFEFE1B92B
:1001F000C0936B00C695C695E09173001E2EE695E0
:10020000E6951E1A1C0EE12DE0937300F0917B0021
:100210001F2EF695F695F6951F1AC6951C0EF12D14
:10022000F0937B00EF1BE2302CF0C298F3E0F093E8
:10023000830005C0F0918300FF2309F4C29AC0E057
:1002400028C0C0E0E0E0EC0FE7B923C0D03049F4AB
:10025000F2E0E0E0EF0FE7B9C0937000C0937800E0
:1002600018C0D23049F4F3E0E0E0EF0FE7B9C093F3
:100270007200C0937A000DC0D33019F7F0E0E0E0CF
:10028000EF0FE7B9C0937300C0937B00EE27E093B4
:100290006000EE27EDBDECBD1895189518951895E2
:00000001FF
